:04000000B6017929A3
:10000800080098181812181664008C1E08281A0878
:1000180003147429040864000C1E0F2899000314A3
:100028007429B616B61EB612B6191E28B6156D2056
:1000380003185B280830A3008120A20DA30B2028F9
:10004800B61E66208B208720B61A5B206020220807
:10005800031074293617361F3613A4002908031D08
:100068003828361B5B287429251883172408840030
:1000780000088313462003187429A40AA903322808
:10008800B616B61EB61236194E28FE39B700361502
:1000980003107429361A5628A60036166D20031840
:1000A8005B282608742003185B28B61E742966206E
:1000B8008B2036113612B6113A0884003808841796
:1000C80080046C283A088400380980058417800564
:1000D800080060208B20662087203708B619013871
:1000E800A2000830A300A20D03186020031C66209C
:1000F8008B208720A30B772860208B203A08840068
:1001080038080005FF3E3B088400390969283B0888
:10011800840039086328A4002908031974296F2169
:10012800A000251883172408840020088000831362
:10013800A40AA9039028B71329080319B71704308C
:10014800A800250EAC202508AC20240EAC202408DD
:100158000F39F63E0318073E0A3EB228A000A8034E
:100168000319B71329080319BC2828020318080023
:100178002008031DB713B71B0800303E6F2908304D
:10018800A600A7003B088400390837191021371D3D
:1001980012213A08840038081521A001A101260877
:1001A80003197429B71807213A088400000838058C
:1001B800FF3EA00DA10DB71C0721A60BD6282708C6
:1001C80037183E29200874290830A6003B08840007
:1001D800390837191021371D12213A0884003809C7
:1001E800192126080319742937183E213A08840072
:1001F800A10CA00C00083804031C38068000072155
:10020800A60BFA2874293B088400390880060000E8
:100218000D290E298006080080041829FF3A800558
:100228001929841780047429FF3A841780057429D2
:10023800A301A200FF30A207031CA307031C742913
:100248000330A100E4302A211E29A101F63EA000B6
:10025800A109031C3529FE300000A0070318302926
:10026800A0076400A10F2F29000020183B2920189F
:100278003D290800A201A3014529A10CA00CA20D4B
:10028800A30DFF3E031841292308A1002208A0005E
:1002980074290310A00DA10DFF3E03184D29200855
:1002A8007429A101A301A20001305F29A101A301C2
:1002B800A20004305F29A80023082102031D662933
:1002C80022082002043003180130031902302805DF
:1002D800031DFF307429840031088A003008820029
:1002E80083130313831264000800831607309900F0
:1002F80020309800831290309800831607309F00B2
:100308000714871007118712C901C3018312FC0162
:10031800FD010130A300F4308A011D2153308A0108
:100328000F2074308A010F2061308A010F2072304B
:100338008A010F2074308A010F200A308A010F20A9
:100348000D308A010F208A110A125E2D8716831636
:10035800FF30C1000A30BF0083128A110A126424D8
:10036800871232308A011C2183164030BE00953036
:10037800C000831283163E08C10007308312BA00FA
:100388000430B8000730BB000230B9000130B700B4
:10039800831641088312A000A1018A01E820831670
:1003A800C1010430BF0083128A110A126424831623
:1003B8004008C10007308312BA000430B800073083
:1003C800BB000230B9000130B70083164108831220
:1003D800A000A1018A01E82083160130BD00831224
:1003E8008A110A126B22871632308A011C21871261
:1003F800640083164A08003C8A110A128312031902
:10040800482A87168316FF30C10007308312BA00C6
:100418000430B8000730BB000230B9000130B70023
:10042800831641088312A000A1018A01E8208A11DD
:100438000A12E024871283164130C1000730831264
:10044800BA000430B8000730BB000230B9000130F0
:10045800B700831641088312A000A1018A01E82091
:100468008316C1010430BF0083128A110A12642462
:100478008316FF30C10083128A110A12BD248A1123
:100488000A12E0248A01FC298316FF30C100493092
:1004980083128A010F204E308A010F2049308A01C9
:1004A8000F2054308A010F2020308A010F204F304E
:1004B8008A010F204B308A010F2021308A010F203A
:1004C8000A308A010F200D308A010F2008006400CD
:1004D80083164A083D028A110A1283120319842AD4
:1004E8000730BA000130B8000730BB000230B9004D
:1004F800B7018A01C3208316CA0083128A016B2AB6
:10050800080087168316FF30BA0083128A110A1270
:10051800CE248A110A12E024871283165830B600B6
:1005280083127F088316B70083127E088316B800EB
:100538002B08B9002A08BA0083128A110A128A24E1
:100548008316FF30BA0083128A110A12CE248A1148
:100558000A12E0248316BD0183128A016B228316D6
:10056800FE30BA0083128A110A12CE2483162E088E
:100578008312FC0083162F088312FD007C08A0005C
:100588007D08A100831631088312A3008316300862
:1005980083128A0157218A110A12031D012B073081
:1005A800BA001030B8000730BB000830B900A030DE
:1005B8008A0146207D088A0146207C088A01462057
:1005C8008A0115208316C10007308312BA0004304F
:1005D800B8000730BB000230B9000130B7008316FD
:1005E80041088312A000A1018A01E820FC0A03192E
:1005F800FD0A8A110A12031DC22A8316FF30C100A0
:100608000230BF0083128A110A1264248A110A1266
:10061800E0240F3083164A05CC0083128A110A128F
:10062800E024640083164A08003C8A110A128312E7
:10063800031D2E2B0730BA000130B8000730BB006D
:100648000230B900B7018A01C3208316CA00831299
:100658008A01152B8A110A121E2408008716831690
:10066800FF30BA0083128A110A12CE248A110A12A4
:10067800E024871283165130B60083127F08831650
:10068800B70083127E088316B8002B08B9002A0821
:10069800BA0083128A110A128A248316FF30BA001C
:1006A80083128A110A12CE248A110A12E0248316B0
:1006B800BD0183128A016B228316FE30BD008312AE
:1006C8008A016B2283162E08AC002F08AD00831216
:1006D80083162C088312A00083162D088312A1000C
:1006E800831631088312A3008316300883128A0107
:1006F80057218A110A12031DB22B0730BA000130A4
:10070800B8000730BB000230B900B7018A01C32026
:100718008316C10007308312BA001030B8000730C2
:10072800BB000830B900A0308A01462083162D0886
:1007380083128A01462083162C0883128A014620D8
:100748008316410883128A0144208316AC0A0319D0
:10075800AD0A8A110A128312031D6C2B8A110A1220
:10076800E0248A110A12E0248A110A121E240800C1
:1007780083165030BE00FF30C00083128A110A125F
:10078800E323080083166030BE0083128A110A1220
:10079800E323080083166130BE0083128A110A120F
:1007A800E323080083160130C3006630BE008312BD
:1007B8008A110A12E3238316C301831208008716DD
:1007C8008316FF30BA0083128A110A12CE248A11C6
:1007D8000A12E024871283163E08B60083127F08A7
:1007E8008316B70083127E088316B8002B08B90059
:1007F8002A08BA0083128A110A128A248316FF3043
:10080800C1000230BF0083128A110A1264248A11BF
:100818000A12E024640083164308013C8A110A1274
:100828008312031D182C08008316BD0183128A0148
:100838006B22080087168316FF30C1000730831229
:10084800BA000430B8000730BB000230B9000130EC
:10085800B700831641088312A000A1018A01E8208D
:100868008A110A12E024871283164D30BA008312C7
:100878008A110A12CE248316C1010430BF008312E4
:100888008A110A1264248316FF30BA0083128A116F
:100898000A12CE240730BA000130B8000730BB0076
:1008A8000230B900B70110308A01C4208316B200A3
:1008B800831221088316B3003208C9008312080086
:1008C80083160130CC008312640083164C083F0263
:1008D8008A110A128312031C892C0730BA000430CB
:1008E800B8000730BB000230B9000130B7008316EA
:1008F80041088312A000A1018A01E8208316CC0ACE
:100908008A110A128312031D682C08000730BA00E6
:100918000430B8000730BB000230B9000130B7001E
:10092800831636088312A000A1018A01E820073047
:10093800BA000430B8000730BB000230B9000130FB
:10094800B700831637088312A000A1018A01E820A6
:100958000730BA000430B8000730BB000230B900D5
:100968000130B700831638088312A000A1018A015C
:10097800E8200730BA000430B8000730BB00023066
:10098800B9000130B700831639088312A000A1010D
:100998008A01E8200730BA000430B8000730BB00ED
:1009A8000230B9000130B70083163A088312A0005C
:1009B800A1018A01E82008000730BA000130B80018
:1009C8000730BB000230B900B7018A01C320831683
:1009D800CA008312080044308A010F2061308A015E
:1009E8000F2074308A010F2061308A010F202030D7
:1009F8008A010F2066308A010F2072308A010F2089
:100A08006F308A010F206D308A010F2020308A0153
:100A18000F204D308A010F204D308A010F204330BE
:100A28008A010F200A308A010F200D308A010F2019
:100A380083162E08AC002F08AD00831283162C08ED
:100A48008312A00083162D088312A1008316310893
:100A58008312A3008316300883128A0157218A1152
:100A68000A12031D5D2D0730BA001030B800073098
:100A7800BB000830B900A0308A01462083162D0833
:100A880083128A01462083162C0883128A01462085
:100A98008A0115208316C100410883128A010F209C
:100AA8008316AC0A0319AD0A8A110A128312031DB0
:100AB800222D08008A01AA21FE01FF018316AA013E
:100AC8000230AB0083128A01BC238316AE01AF014A
:100AD800FF30B0000130B10083128A110A12742D60
:100AE80057308A010F2061308A010F2069308A014E
:100AF8000F2074308A010F2069308A010F206E3070
:100B08008A010F2067308A010F202E308A010F20BA
:100B18002E308A010F200A308A010F200D308A01F9
:100B28000F2011308A010F2011308A010F20113057
:100B38008A010F208A010520403C8A110A12031DF0
:100B48009E2D0B30A9000530B000B101A501A030E1
:100B58008A018F2013308A010F2013308A010F2059
:100B68008316C601831264000B30831646028A116D
:100B78000A1283120318FF2D83164608A03E84002C
:100B880000088312B200FF30A200A20A22080F3C1C
:100B98008A110A12031CF32D8A110A12DF25320268
:100BA8008A110A12031DC92D22088316C400831254
:100BB8008A110A12F32D05308A0022088207303480
:100BC80031343234333434343534363437343834D9
:100BD800393441344234433444344534463483163A
:100BE8004608A03E840044088000C60A8A110A12FA
:100BF8008312031DB72D83162008C800210883120D
:100C0800A000A10104308A015021B2002108B300DC
:100C180083162208831232048316BB00230883122A
:100C2800A000A10104308A015021B2002108B300BC
:100C38008316240883123204FF00831625088312C2
:100C4800A000A10104308A015021B2002108B3009C
:100C58008316260883123204FE008316270883129F
:100C6800A000A10104308A015021B2002108B3007C
:100C780083162808831232048316AB0029088312CE
:100C8800A000A10104308A015021B2002108B3005C
:100C980032088316AA0464003B08003C8A110A1231
:100CA8008312031D5B2E83160130BB008312640080
:100CB80083164808003C8A110A12831203198A2EE7
:100CC800640083164808013C8A110A12831203192A
:100CD800372F640083164808023C8A150A128312CB
:100CE80003190328640083164808033C8A150A126E
:100CF80083120319A228640083164808043C8A1545
:100D08000A1283120319A4288A01952D11308A0129
:100D18000F2041308A010F2064308A010F2064308F
:100D28008A010F2072308A010F203A308A010F2081
:100D38000430A9007E08A4007F08A5000E30B0008A
:100D4800B1018A019F200430A90083162A08831262
:100D5800A40083162B088312A5000E30B000B10141
:100D68008A019F200A308A010F200D308A010F2046
:100D780013308A010F2083160130BC0083126400EF
:100D880083163C083B028A110A128312031C352F72
:100D98008A01322383162E08AC002F08AD00831277
:100DA80083162C088312A00083162D088312A10035
:100DB800831631088312A3008316300883128A0130
:100DC80057218A110A12031D1E2F0730BA0010304E
:100DD800B8000730BB000830B900A0308A014620AF
:100DE80083162D0883128A01462083162C08831245
:100DF8008A0146208A0115208316C100113083120A
:100E08008A010F200230A900831641088312A4002A
:100E1800A5010E30B000B1018A019F2013308A016C
:100E28000F208316AC0A0319AD0A8A110A1283121D
:100E3800031DD42E00308316AA0702300318013E82
:100E4800AB0764008A110A128312031C2E2FFE0AB4
:100E58000319FF0A8316BC0A8A110A128312031D9A
:100E6800C32E8A01952D11308A010F2041308A0145
:100E78000F2064308A010F2064308A010F207230FD
:100E88008A010F203A308A010F200430A9007E0819
:100E9800A4007F08A5000E30B000B1018A019F2090
:100EA8000430A90083162A088312A40083162B088D
:100EB8008312A5000E30B000B1018A019F200A30CC
:100EC8008A010F200D308A010F2013308A010F206C
:100ED80083160130BC008312640083163C083B0271
:100EE8008A150A128312031C01288A0132238316E9
:100EF8002E08AC002F08AD00831283162C0883122D
:100F0800A00083162D088312A100831631088312CE
:100F1800A3008316300883128A0157218A110A1206
:100F2800031DEA2F0730BA001030B8000730BB00A5
:100F38000830B900A0308A01462083162D08831294
:100F48008A01462083162C0883128A0146208A01CA
:100F580015208316C100640041080A3C8A110A1250
:100F680083120319D62F6400831641080D3C8A1199
:100F78000A1283120319D62F831641088312A00080
:100F88007E308A015521B200831641088312A000E1
:100F980020308A015A21B400320834048A110A1216
:100FA800031DE12F11308A010F2083164108831297
:100FB8008A010F2013308A010F208316AC0A031907
:100FC800AD0A8A110A128312031D812F003083167D
:100FD800AA0702300318013EAB0764008A110A12FF
:100FE8008312031CFA2FFE0A0319FF0A8316BC0A90
:100FF8008A110A128312031D702F8A01952D8316F8
:101008000130BC008312640083163C083B028A1539
:101018000A128312031C76288316AC01AD01013035
:10102800C600831264000930831646028A150A1224
:10103800831203185D2811308A010F204030A9005F
:101048000530B000B101A5013C308A018F20133072
:101058008A010F2013308A010F2013308A010F20D4
:1010680013308A010F200730BA001030B80007305B
:10107800BB000830B900A0308A01462083162D082D
:1010880083128A01462083162C0883128A0146207F
:101098004030A900A5013C308A012E20403083163B
:1010A800AC070318AD0AC60A8A150A128312031D73
:1010B80016288A01852200308316AA0702300318F1
:1010C800013EAB0764008A150A128312031C6F28BD
:1010D800FE0A0319FF0A8316BC0A8A150A1283122C
:1010E800031D072811308A010F2044308A010F2080
:1010F80061308A010F2074308A010F2061308A0123
:101108000F2020308A010F2057308A010F207230BB
:101118008A010F2069308A010F2074308A010F205C
:1011280074308A010F2065308A010F206E308A01E1
:101138000F2013308A010F208A01952D8A01952DE1
:101148008A01952D8A01952D63008A150A12A8280F
:02400E003D3D36
:00000001FF
